:1000000012C02AC029C028C027C094C026C024C05E
:1000100023C022C021C020C01FC01EC01DC01CC0E4
:100020001BC01AC019C011241FBECFEDCDBF10E0F8
:10003000A0E6B0E0E0E4F6E002C005900D92A03644
:10004000B107D9F710E0A0E6B0E001C01D92A636D6
:10005000B107E1F777D1F2C2D3CF1F920F920FB65B
:100060000F9211248F9380916000813418F01092C8
:100070006000909A80916000882329F4809161004B
:10008000882309F041C080916000843029F4809178
:100090006100882309F042C080916000883021F41B
:1000A00080916100823080F5809160008C3021F475
:1000B00080916100823090F580916000803121F460
:1000C00080916100833000F580916000843121F4DB
:1000D00080916100833010F580916000883121F4B7
:1000E00080916100843080F4809160008C3121F433
:1000F00080916100843090F480916000833231F40B
:1001000080916200813011F4909809C08091600064
:10011000873329F480916200813009F4909A8091AC
:1001200060008F5F809360008F910F900FBE0F90E3
:100130001F9018951F920F920FB60F9211248F9354
:100140009F93809164009091650001969093650063
:10015000809364009F918F910F900FBE0F901F901E
:10016000189592B3880F880F880F9776982B92BBBB
:100170008AE18A95F1F708951DBC1CBC10926500B8
:1001800010926400089580EF87BB80E293E028EC32
:1001900030E0F9013197F1F70197D9F780916300C9
:1001A00090E028EC30E040EF09C018BAF90131972F
:1001B000F1F748BBF9013197F1F79F5F9817A8F362
:1001C00090E048EC50E013C0909828EE33E0FA013C
:1001D0003197F1F721503040D1F7909A24EC39E073
:1001E000FA013197F1F721503040D1F79F5F98170E
:1001F00058F317BA8E5F809363008A3018F083E05B
:100200008093630020916300E199FECF1CBA82E0E5
:1002100090E08EBB2DBB0FB6F894E29AE19A0FBE28
:1002200088E893E128EC30E0F9013197F1F7019784
:10023000D9F7089580EF87BB80E588BB82B38776C6
:1002400082BB9AE1892F8A95F1F726B382B387762C
:10025000886082BB9A95F1F7B39B02C022E005C08B
:100260002695269526952095217082B38776806104
:1002700082BB8AE18A95F1F7B39B23E082B387764C
:10028000886182BB8AE18A95F1F7B39924E080EA1C
:1002900088BB82B3877682BB8AE18A95F1F7B399EE
:1002A00021E082B38776886082BB8AE18A95F1F784
:1002B000B39B22E082B38776806182BB8AE18A9514
:1002C000F1F7B39923E082B38776886182BB8AE134
:1002D0008A95F1F7B39B24E017BA8699FECF48ECD4
:1002E00050E0222399F428EC30E0909888EE93E0D7
:1002F000F9013197F1F70197D9F7909A88E293E2E3
:10030000F9013197F1F70197D9F7EFCF30E09098E5
:1003100088EE93E0FA013197F1F70197D9F7909AB7
:1003200080EA9FE0FA013197F1F70197D9F73F5F33
:10033000321768F380E197E2FA013197F1F70197FC
:10034000D9F7CFCFDF92EF92FF920F931F93DF93F6
:10035000CF93CDB7DEB72C970FB6F894DEBF0FBEA4
:10036000CDBF17BA89E181BB80EF88BB81E682BB34
:10037000E199FECF81E090E0982F8EBBE09A8DB39B
:100380008438E1F0E199FECF1CBA9EBB84E88DBBB6
:100390000FB6F894E29AE19A0FBE83E0809363006F
:1003A000E199FECF1CBA82E090E08EBB83E08DBB6A
:1003B0000FB6F894E29AE19A0FBE09C0E199FECF18
:1003C00082E090E08EBBE09A8DB380936300859BC2
:1003D00031DF869BD8DE19821D8219861A821E8221
:1003E0001A861B821F821B861C8218861C8688EE3A
:1003F00093E028EC30E0F9013197F1F70197D9F754
:1004000085E083BF81E08EBD82E889BF78941DBC02
:100410001CBC10926500109264008E010B5F1F4F90
:10042000FF24F394DE011996BE016F5F7F4FEAE16E
:10043000EE2E80916400909165000A9709F49098DF
:100440008091640090916500449709F5909A10920C
:100450006500109264001BC020E030E086B390E09D
:100460002C5F3F4F022E02C0959587950A94E2F7C4
:100470002450304080FF02C0FD0101C0F801E20FAE
:10048000F31FF0822F5F3F4F2430310539F7809101
:100490006400909165000397F8F220E030E0F801E5
:1004A000E20FF31F8081813051F4FD01E20FF31F51
:1004B0008081813021F4FB01E20FF31F80832F5FE5
:1004C0003F4F2430310559F740E050E0942FFB01B5
:1004D000E40FF51F8081813021F582B39A0153E04A
:1004E000220F331F5A95E1F78776822B82BB8E2D20
:1004F0008A95F1F79F5F909361009150933609F4CC
:1005000098CF242FA5E0EA2EF12CEC0EFD1E31E051
:100510008E01075F1F4FDD24D394DE0111967AE12F
:1005200006C04F5F5F4F4430510581F682CF19827C
:100530001D8219861A821E821A861B821F821B86C2
:100540001C8218861C861DBC1CBC10926500109273
:1005500064001BC040E050E086B390E04C5F5F4F0A
:10056000042E02C0959587950A94E2F744505040B6
:1005700080FF02C0F80101C0F701E40FF51F3083CE
:100580004F5F5F4F4430510539F78091640090917F
:1005900065000397F8F240E050E0F701E40FF51F23
:1005A0008081813051F4F801E40FF51F80818130A2
:1005B00021F4FD01E40FF51F80834F5F5F4F44304E
:1005C000510559F78981882381F48A81882369F448
:1005D0008B81882351F48C81882339F4233629F0C8
:1005E000D09262001092610023E640E050E0642F58
:1005F000FD01E40FF51FE081E130B1F4942F82B3E7
:10060000F3E0440F551FFA95E1F78776842B82BB00
:10061000872F8A95F1F7261711F0E09362009F5F0C
:1006200090936100262F05C04F5F5F4F4430510506
:10063000F1F686997CCF1092620079CFF894FFCFC3
:00000001FF
